:100000000C945E000C9486000C9486000C94860080
:100010000C9486000C9486000C9486000C94860048
:100020000C9486000C9486000C9486000C94860038
:100030000C9486000C9486000C9486000C94860028
:100040000C946E160C9486000C94FF170C943118C7
:100050000C9486000C9486000C9486000C94860008
:100060000C9486000C948600000000080002010039
:100070000003040700000000000000000102040863
:100080001020408001020408102001020408102002
:10009000040404040404040402020202020203032E
:1000A0000303030300000000250028002B000000CC
:1000B0000000240027002A00BA06611811241FBE80
:1000C000CFEFD8E0DEBFCDBF11E0A0E0B1E0E6E4C5
:1000D000F4E302C005900D92AC3AB107D9F723E0E2
:1000E000ACEAB1E001C01D92AE30B207E1F710E01A
:1000F000CCEBD0E004C02297FE010E94161AC83B48
:10010000D107C9F70E94F9180C94211A0C94000029
:1001100080E00895089580E0089581E008950895AD
:1001200080910A0190910B01A0910C01B0910D01F9
:10013000843F21E09207A105B10524F4C296A11DD8
:10014000B11D04C082E390E0A0E0B0E080930A011A
:1001500090930B01A0930C01B0930D0108950895A5
:100160000895860F911D860F911DFC0156874587C6
:1001700081E00895CF93DF93EC018C819D81DC01B8
:10018000ED91FC910480F581E02D6E8109951F862B
:10019000188A81E08A8B1E821B8A1C8A1D8A1E8A0D
:1001A0001F8A80E0DF91CF910895FC018681089538
:1001B00081E0633009F080E0089581E0623009F069
:1001C00080E00895860F911D860F911DFC018585A5
:1001D00096850895FC0187890895EF92FF92CF9349
:1001E000DF93FC01E7012289223029F16787408BE8
:1001F0008B8183708330F9F48A8187FF1CC08E81E4
:10020000908D981708F4808F822F90E0DC01AA0F60
:10021000BB1FA80FB91FAE0FBF1F8A818F70179623
:100220008C9317978C8118968C93189784E0199665
:100230008C932F5F228BDF91CF91FF90EF900895E9
:10024000EF92FF920F9302970E94ED000F91FF90A3
:10025000EF900895089561E080910E010C94C91704
:1002600060E080910E010C94C9170F931F93CF93F8
:10027000DF93EB018981992787FD909597FF03C054
:1002800091958195910960910601709107010E94F5
:10029000001A6F5F7F4F70935A026093590200E01B
:1002A00010E08091590290915A02081719070CF03A
:1002B00068C02981332727FD3095809108019091EE
:1002C00009018217930734F561E0809114010E94BF
:1002D000C91780910A0190910B010E94211761E0DA
:1002E000809112010E94C91780910A0190910B011F
:1002F0000E94211760E0809114010E94C91780912B
:100300000A0190910B010E94211760E08091120177
:100310000E94C9172981332727FD30958091080154
:10032000909109019195819591092817390734F524
:1003300061E0809112010E94C91780910A01909199
:100340000B010E94211761E0809114010E94C917DE
:1003500080910A0190910B010E94211760E0809129
:1003600012010E94C91780910A0190910B010E940D
:10037000211760E0809114010E94C9170F5F1F4F81
:1003800090CF8A81992787FD909597FF03C091951B
:100390008195910960910601709107010E94001AF0
:1003A0006F5F7F4F709358026093570200E010E038
:1003B0008091570290915802081719070CF068C0F5
:1003C0002A81332727FD30958091080190910901FA
:1003D0008217930734F561E0809110010E94C917DC
:1003E00080910A0190910B010E94211761E0809198
:1003F0005B020E94C91780910A0190910B010E9433
:10040000211760E0809110010E94C91780910A01B4
:1004100090910B010E94211760E080915B020E9485
:10042000C9172A81332727FD3095809108019091C3
:1004300009019195819591092817390734F561E0F3
:1004400080915B020E94C91780910A0190910B0173
:100450000E94211761E0809110010E94C9178091CC
:100460000A0190910B010E94211760E080915B02CC
:100470000E94C91780910A0190910B010E942117D7
:1004800060E0809110010E94C9170F5F1F4F90CF4D
:10049000DF91CF911F910F9108952F923F924F922C
:1004A0005F926F927F928F929F92AF92BF92CF9204
:1004B000DF92EF92FF920F931F93CF93DF9300D0C1
:1004C00000D0CDB7DEB76C017C836B835A83498340
:1004D0004C0180E1880E911C5601A7E0AA0EB11CC8
:1004E00011E044E0442E57E0352E3601B2E16B0EA8
:1004F000711C63E0262E72E0572E8B819C81892B24
:1005000009F412C1F60180A1823061F128F4882338
:1005100049F0813079F0F1CF833041F1843009F432
:100520004BC0EBCF5482858196819087878352861A
:10053000518610A3AE014D5F5F4FBE016F5F7F4FCD
:10054000C5010E942D12882309F4EEC0D60115962C
:10055000ED91FC911697808191968C939197818172
:1005600092968C93F6017682658220A2D6019296AD
:100570008C91843081F018F4823079F014C0853089
:1005800081F0813281F4D60191968C9191978250BD
:1005900014968C9308C0F60113A2D60114963C92CF
:1005A00002C0F6018483F601858196819087878356
:1005B00084818287818740A2D60192968C91843073
:1005C000B1F0853009F442C0823009F06EC0AE014E
:1005D0004D5F5F4FBE016F5F7F4FC5010E942D12BF
:1005E000882309F4A1C0F601858984A38EC0AE01D9
:1005F0004D5F5F4FBE016F5F7F4FC5010E942D129F
:10060000882309F491C0D60155968C915597833073
:1006100009F07BC056968C915697813009F075C0D1
:1006200098969C91989757968C91992321F08823BE
:1006300009F46BC003C0823009F067C0F60113A350
:10064000928996A3938997A385A35FC0AE014D5F5E
:100650005F4FBE016F5F7F4FC5010E942D1288233F
:1006600009F462C0D60193968C919397882309F47C
:100670004CC012968D919C911397009709F445C038
:10068000DC01ED91FC910190F081E02D7401D60127
:1006900095960C91959797962C91979796964C9145
:1006A000969794966C91099530C0F60181A1958535
:1006B000992319F0913031F023C090E00297978789
:1006C000868715872B813C8189819A81782F692FB4
:1006D000D6011E964D915C911F9741155105E9F089
:1006E00001962115310541F041505109F601578716
:1006F000468721503109EACF79836A831C821B82A5
:10070000F60186859785892B79F4D60116969C92F9
:100710008E92159790961C92F0CE9A8389833C8393
:100720002B83F6011586ECCF0F900F900F900F9052
:10073000DF91CF911F910F91FF90EF90DF90CF90BD
:10074000BF90AF909F908F907F906F905F904F90F1
:100750003F902F9008959FB7F89420916602809162
:100760006402213019F48DBB9FBF08958FBF089597
:10077000CF92DF92EF92FF920F931F93CF93DF936D
:10078000CDB7DEB762970FB6F894DEBF0FBECDBF10
:100790006C01DC0157968C91882369F00E94B81691
:1007A000F6010389148925893689601B710B820B38
:1007B000930B97FF02C0F12C39C0F601838590E0BE
:1007C0009A8B898BE12C8E010F5F1F4F9E012F5E4C
:1007D0003F4F42856681848195810E94400EF82EAC
:1007E000811118C029893A892330310598F0D60142
:1007F0001D968D919C911E97009761F0DC01ED9103
:10080000FC910190F081E02D8E010F5F1F4F40E0C1
:10081000B60109950E94B816F601208D620F711D70
:10082000811D911D638B748B858B968B8F2D6296AA
:100830000FB6F894DEBF0FBECDBFDF91CF911F91F1
:100840000F91FF90EF90DF90CF9008953F924F92DD
:100850005F926F927F928F929F92AF92BF92CF9250
:10086000DF92EF92FF920F931F93CF93DF93CDB759
:10087000DEB7EB970FB6F894DEBF0FBECDBF7C019D
:10088000462E342E522EDC011496AD90BC90159756
:1008900016968C911697811111C158961C92D5010C
:1008A000ED91FC910190F081E02D60E0C50109958A
:1008B0006C01009711F486ED0BC1FC0180809180E2
:1008C0008114910409F4FCC03701F7E06F0E711C2C
:1008D000DC0111967C926E9214965C928E01065DFC
:1008E0001F4F28E030E040E060E0F701848195810F
:1008F0000E943F0D182F8111E7C01AA5D6018D92D5
:100900009C92D501ED91FC910280F381E02D232D85
:1009100040E0642DC5010995F7018683882309F419
:10092000D1C099A99087282F40E060E0848195810B
:100930000E94EC0D982ED501ED91FC91D6011496F4
:100940001C92882361F00480F581E02DD701169672
:100950006C91C5010995F7011682892DB9C00190E6
:10096000F081E02DD70116966C91C501099500978D
:1009700009F4A1CF133108F012E1FC0154821111E6
:100980000FC04BAC512CEDE2AE2EE1E0BE2E470184
:10099000F2E08F0E911C6E0181E1C80ED11C39C0AE
:1009A000212F30E08E01065D1F4F40E0D7011696E3
:1009B0006C91169714968D919C9115970E943F0DFE
:1009C000182F811171C0DDCFBA82A9829C828B82DF
:1009D0001E86188A1F8619A21AA21BA219A6DF82D8
:1009E000CE82D986C8868D818B878A87DD86CC8624
:1009F0008E010F5F1F4F252D40E0F7016681848136
:100A000095810E948D0DD70152968C91823019F0FC
:100A100053945410D9CFF7018289823009F043C032
:100A2000930142E06681848195810E948D0868EE81
:100A300073E080E090E00E94E716D7011F962C91AA
:100A40001F9740E016966C91169714968D919C9185
:100A500015970E941B0E182F811126C068EE73E0B7
:100A600080E090E00E94E71640E060E0C7010E944D
:100A7000A011182F811118C020E040E060E0C701EC
:100A80000E94761183E391E09A838983AE014F5FE0
:100A90005F4F60E070E0C7010E94331181E0F70111
:100AA000878B80E015C011EDD701ED91FC9104809A
:100AB000F581E02DC7010995812F0AC089ED08C095
:100AC00087ED06C084ED04C0F60191828082ECCFF0
:100AD000EB960FB6F894DEBF0FBECDBFDF91CF917E
:100AE0001F910F91FF90EF90DF90CF90BF90AF904C
:100AF0009F908F907F906F905F904F903F90089560
:100B000020916602222399F03FB7F8942091660263
:100B1000213059F42DB3209364024DB32091650226
:100B2000209524232DBB3FBF02C0309364028CBDAF
:100B30009DBD089580EE91E00C943A102A9A089594
:100B4000CF93C82F80E591E00E9480052A98CEBD02
:100B500000000DB407FEFDCF8EB51EBC00000DB425
:100B600007FEFDCFCEB50E949E05809166028111E1
:100B70000E94AB038C2FCF9108951F93CF93DF93E7
:100B80001F92CDB7DEB7182F80E591E069830E94F0
:100B900080052A98812F82608EBD69810DB407FE81
:100BA000FDCF8EB56EBD0DB407FEFDCF8EB50E9494
:100BB0009E0580916602882331F00F90DF91CF91DE
:100BC0001F910C94AB030F90DF91CF911F9108956B
:100BD00088EF0E94A005807C8034A1F018F488235F
:100BE00001F10895803819F0803CB9F0089588ED3E
:100BF0000E94A00581FD0BC069EC88ED0E94BD0537
:100C000082E00CC088ED0E94A00581FDF5CF6BEC61
:100C100088ED0E94BD0583E001C081E08093AC01B6
:100C2000089561ED88ED0E94BD051092AC01089514
:100C30000F931F93CF93DF938C01229A0E949E05FE
:100C40000E943816229A0E949E05219868E188E841
:100C50000E94BD0560E288E70E94BD0560E088E76C
:100C60000E94BD05C0E0D0E088E60E94A005219664
:100C700080FD06C0CF3F8FEFD807B1F78FEF1DC0C3
:100C800061EC88ED0E94BD0560E680ED0E94BD0527
:100C900064E088EE0E94BD0588EE0E94A00582FFF8
:100CA000FBCFC8010E94E80560E288EC0E94BD0508
:100CB00061E080E80E94BD0580E0DF91CF911F9147
:100CC0000F91089561E0809114010E94901761E0F6
:100CD000809112010E94901761E0809110010E94A2
:100CE000901761E080915B020E94901761E0809113
:100CF0000E010E94901780EE91E00E9418068F3F2F
:100D000031F466E171E081E792E00E94E61868EC58
:100D100070E080E090E00E94E7160E94B8166857E5
:100D20007C4E8F4F9F4F6093B2017093B3018093BD
:100D3000B4019093B5018DEA91E09093C401809342
:100D4000C30160E0809114010E94C91760E08091A6
:100D500012010E94C91760E0809110010E94C9171A
:100D600060E080915B020E94C91761E080910E01F2
:100D70000C94C91780EE91E00E944B0760EE71E081
:100D80008FEC91E00E94C41480EE91E09093BB013F
:100D90008093BA018DE491E09093B7018093B601FE
:100DA0008BE691E09093B9018093B8011092C9014C
:100DB0001092CA011092CB011092CC011092CD0179
:100DC0001092BD0188E08093BE018CE38093BF0147
:100DD0001092C0011092C10184E08093C20181E0B1
:100DE0008093C8011092C7011092C5011092C401EE
:100DF0001092C301E6E3F2E080E090E021913191AE
:100E0000232B51F4FC01EE0FFF1FEA5CFD4F86EB34
:100E100091E09183808304C001968031910571F740
:100E200089E391E09093AE018093AD010895FC01B8
:100E300020812EBDDC019B012150310951F011961A
:100E40005C9111970DB407FEFDCF4EB55EBD4D937D
:100E5000F3CFFB013197E80FF91F0DB407FEFDCF6B
:100E60008EB5808308958EBD00000DB407FEFDCFC2
:100E70008EB5089580916602882361F09FB7F8943B
:100E80002091660280916402213019F48DBB9FBFCE
:100E900008958FBF0895FC0181E791E091838083DD
:100EA0001582108681E0818712869F012E5F3F4F59
:100EB00037832683128288E083838CE3848380E0F7
:100EC00090E041E0DF01A80FB91F1D961C921D970D
:100ED0001E964C931E971F961C921F971C963C9330
:100EE0002E931B9705968B34910561F7EA58FF4FB7
:100EF000108281E1809361020895CF92DF92EF9298
:100F0000FF920F931F93CF93DF931F92CDB7DEB75E
:100F10007C016623B1F18C01C12CD12CF801EA5A75
:100F2000FF4F80819181009719F1DC01ED91FC91D7
:100F30000084F185E02D698309956981861318C0C5
:100F4000F601BB96EE0FFF1FEE0DFF1D8081918114
:100F5000DC01ED91FC910480F581E02D0F90DF9193
:100F6000CF911F910F91FF90EF90DF90CF90099458
:100F7000BFEFCB1ADB0A0E5F1F4FE0E1CE16D104A4
:100F800069F680E00F90DF91CF911F910F91FF9054
:100F9000EF90DF90CF90089520E030E041E0FC0139
:100FA000E20FF31F5585561739F04F5F2B5F3F4F08
:100FB0004031A9F780E00895842F0895EF92FF92C1
:100FC0001F93CF93DF9300D0CDB7DEB77C01162FF0
:100FD00067FD5FC0283008F05CC0442331F0DC01BD
:100FE00015968C91873009F454C060E0C7012A83BC
:100FF00049830E94CC072A814981882309F449C08A
:10100000E82FF0E0111123C085E08E9FD0018F9F63
:10101000B00D1124AE0DBF1D442359F081E4189684
:101020008C93D70115968C9115978F5F15968C939D
:1010300003C081E018968C9385E08E9FD0018F9F2E
:10104000B00D1124AE0DBF1D18968C9123C0612FD9
:101050006770660F660F660F442361F06064D70106
:1010600015968C9115978F5F15968C938770687F76
:10107000682B03C02770687B622B85E08E9FD001B0
:101080008F9FB00D1124AE0DBF1D18966C93862F47
:1010900001C080E00F900F90DF91CF911F91FF90E2
:1010A000EF900895CF93DF93EC01662359F00E94EF
:1010B000CC07882349F09E0145E0849F200D311D17
:1010C0001124C901069602C080E090E0DF91CF9123
:1010D0000895CF93DF931F92CDB7DEB749830E9467
:1010E00052084981009789F0DC01ED91FC9111973C
:1010F000309759F013969C9180E0891731F0208148
:10110000241731F033968F5FF8CF80E090E001C074
:10111000CF010F90DF91CF910895EF92FF921F932F
:10112000CF93DF931F92CDB7DEB7162F790121152C
:10113000310569F049830E945208FC0149810097FA
:1011400041F01283F182E082438380E003C088EDA6
:1011500001C086ED0F90DF91CF911F91FF90EF902E
:1011600008952A9808951F93CF93DF931F92CDB7C8
:10117000DEB7182F80E591E00E9480050E94B1083B
:10118000812F0E94330780E00E94330789830E94E9
:101190009E050E943A0789810F90DF91CF911F91A0
:1011A00008951F93CF93DF9300D01F92CDB7DEB782
:1011B000182F80E591E06B830E9480050E94B108A2
:1011C000126019836B816A8362E070E0CE01019640
:1011D0000E9417070E949E050E943A070F900F90E9
:1011E0000F90DF91CF911F9108958F929F92BF92A0
:1011F000CF92DF92EF92FF920F931F93CF93DF93E3
:101200001F92CDB7DEB74C01B62E690149830E940B
:1012100052087C014981009709F443C0FC01808198
:101220009181892B09F43FC06B2DC4010E9469088C
:10123000F601918380830097C1F1FC0122812695FC
:101240002695822F90E0409764F441E050E060E002
:1012500070E004C0440F551F661F771F2A95D2F710
:1012600002C040E050E841505109F80151834083E9
:101270006B2D80EE0E94D10888ED0E94B308F70123
:101280009481992339F0F401EA58FF4F608162603C
:10129000682B02C0682F697F88ED0E94D10880E02A
:1012A00005C086ED03C087ED01C08BED0F90DF9187
:1012B000CF911F910F91FF90EF90DF90CF90BF9053
:1012C0009F908F9008958F929F92AF92BF92CF92EE
:1012D000DF92EF92FF920F931F93CF93DF931F92B2
:1012E000CDB7DEB7A62E890149830E94B8166B01DF
:1012F0007C0188E8C80E83E1D81EE11CF11C812C1A
:10130000912CB12C20E04981A42A29830E94B8168F
:101310006C197D098E099F09298197FF2DC06A2DBF
:1013200080EF0E94D1080E94B8166C197D098E09C1
:101330009F0997FF09C088EC0E94B30887FFF3CF8D
:1013400060E888EC0E94D10888EF0E94B308282F3B
:101350002F70243019F02E3059F00EC0EFEF8E1A96
:101360009E0A0115110589F28016910671F604C0D6
:10137000B394F3E0BF12C9CF822F0F90DF91CF91CA
:101380001F910F91FF90EF90DF90CF90BF90AF90A3
:101390009F908F9008959F92AF92BF92CF92DF92CD
:1013A000EF92FF920F931F93CF93DF937C01B42EA4
:1013B000122FAA24A394DC01A60FB11DA60FB11D04
:1013C0006D0186E5C80ED11CC42FD0E0AB96CC0FC2
:1013D000DD1FCE0DDF1DD6018D919C91DC01ED91BD
:1013E000FC910280F381E02D202F412F6B2D099578
:1013F000803EC1F4B1100BC061E088EE0E94D108BC
:1014000066E670E080E090E00E94E71615C08881F3
:101410009981DC01ED91FC910284F385E02D612F2F
:1014200009950AC08D3031F48FEF8A0D833008F0B2
:1014300042C017C0811142C0F60180819181DC0158
:10144000ED91FC910190F081E02D202F412F6B2D2B
:101450000995982EBDE08B130CC08FEF8A0D833059
:1014600050F464E670E080E090E00E94E716A394F8
:10147000B2CF882311F1B1100BC061E088EE0E9459
:10148000D10866E670E080E090E00E94E71611C0A7
:10149000EB2DF0E0BB96EE0FFF1FEE0DFF1D8081E0
:1014A0009181DC01ED91FC910284F385E02D612FA7
:1014B0000995892D03C08DE001C080E0DF91CF91B7
:1014C0001F910F91FF90EF90DF90CF90BF90AF9062
:1014D0009F9008950F931F93CF93DF93D82FC62F1C
:1014E0008A0180E591E00E9480050E94B1088D2F5D
:1014F00082600E943307D0E0209721F0BE01C8012E
:101500000E941707C00FD11F0E949E050E943A0734
:10151000CE01DF91CF911F910F9108952F923F92AD
:101520004F925F926F927F928F929F92AF92BF92F3
:10153000CF92DF92EF92FF920F931F93CF93DF939F
:1015400000D000D01F92CDB7DEB77D836C835A01E7
:101550006901FB0121808FEF820D803408F06FC09C
:101560000E94B8162B013C01F8E84F0EF3E15F1E14
:10157000611C711CEC81FD81828180FF02C060E8EA
:1015800001C060E488EE0E94D10820E0312CC11433
:10159000D10409F444C076012C143D0408F471010F
:1015A000EA82A8016E2D80E10E946A0A6E2D88E30E
:1015B0000E94D108EC81FD816081606280EF0E9411
:1015C000D10888EC0E94B30887FFFBCF60E888EC65
:1015D0000E94D10888EF0E94B308282F2F70812C19
:1015E000912C1982222309F46BC02B830E94B81618
:1015F00064197509860997092B8197FF61C0263008
:1016000001F12E3009F456C0243049F4FFEF8F1A4F
:101610009F0AA114B10459F18A149B0441F588EF83
:101620002B830E94B30885FB882780F9EC81FD811C
:10163000928180FB90F992832B81822F46C08AEDA4
:1016400044C088EF0E94B30885FB882780F991E0A9
:101650008927EC81FD81928180FB90F9928390FF34
:1016600002C060E801C060E488EE0E94D10860E03A
:1016700088E30E94D108F801608180E10E94D108CE
:101680006A8188E30E94D108EC81FD8160816062FB
:1016900080EF0E94D10888EC0E94B30887FFFBCF3F
:1016A00060E888EC0E94D10888EF0E94B308282FD8
:1016B0002F7098CF89818F5F89838330C1F6AFCF38
:1016C000CE18DF080E0D1F1D62CF0F900F900F90E8
:1016D0000F900F90DF91CF911F910F91FF90EF909E
:1016E000DF90CF90BF90AF909F908F907F906F9042
:1016F0005F904F903F902F9008952F923F924F927E
:101700005F926F927F928F929F92AF92BF92CF9291
:10171000DF92EF92FF920F931F93CF93DF93CDB79A
:10172000DEB729970FB6F894DEBF0FBECDBF1C0100
:10173000798768875B834A836901D9018D909C9082
:101740001197FB01F181F9831D921C92DB01129626
:101750008C9181FF02C060E201C060E188EE0E94CE
:10176000D1088E2D90E0A0E0B0E08C839D83AE8305
:10177000BF83482C2A813B81A885B9854C9160E0C4
:10178000C1010E946309F82EB6E08B1316C088EFE2
:101790000E94B3088295817091E08927E885F985D8
:1017A000928180FB91F9928391FF02C060E201C0B7
:1017B00060E188EE0E94D108DDCF811166C088EC1F
:1017C0000E94B30882FF5FC080E30E94B308582ED6
:1017D00090E08816990608F4542CD6018D919C91BE
:1017E000652C712CF401E81BF90BCF01F7FF02C047
:1017F00080E090E05301861597050CF45C0180E5CC
:1018000091E00E9480050E94B10888E00E943307A1
:10181000A50160E070E0C8010E941A1AA114B10489
:1018200021F0B501C8010E9417070A0D1B1D0E9477
:101830009E050E943A0764E088EC0E94D108D60118
:101840008D919C911197860D971D8D939C93B981D5
:101850005B1618F08815990560F088EF0E94B308B0
:1018600082958170E885F985928180FB91F9928358
:101870000CC0EE2009F47ECF6C817D818E819F812A
:101880000E94E71677CF30EFF32E8F2D29960FB6F3
:10189000F894DEBF0FBECDBFDF91CF911F910F91A6
:1018A000FF90EF90DF90CF90BF90AF909F908F9080
:1018B0007F906F905F904F903F902F9008952F9260
:1018C0003F924F925F926F927F928F929F92AF92D0
:1018D000BF92CF92DF92EF92FF920F931F93CF931D
:1018E000DF93CDB7DEB762970FB6F894DEBF0FBEB9
:1018F000CDBF3C01F42E322E202E5C2D4FA058A4DB
:10190000C9A4DAA4188A1F861E861D868E01035F6D
:101910001F4F9E01215F3F4F598B0E94F508598947
:10192000811194C039822A82EB825C83BE82AD82AF
:1019300098868F82AE014F5F5F4F68E080E20E9421
:101940006A0A2D853E854F2D60E1C3010E9463091F
:10195000182F81117AC0232C221C2224221CC1148E
:10196000D10409F466C0EF85F8898281222009F448
:1019700053C082608283540133243394A114B10490
:1019800009F455C05C864B864D855E856F857889E8
:10199000E12C86019E01255F3F4FC3010E947D0B14
:1019A000182F8630B1F42F85388988EF298B3A8B30
:1019B0000E94B30885FB882780F9832529893A8905
:1019C000D90112969C91129780FB91F912969C93E3
:1019D000D5CF81113AC0EBA5FCA53097A1F00190BD
:1019E000F081E02D0190F081E02DC4018A199B095E
:1019F0009A8789876B857C859E01275F3F4FA6016B
:101A00008BA59CA509958B859C85A81AB90A841578
:101A1000950508F0B3CF0DC0816082834D855E854A
:101A200086019201BF01C3010E948E0A182F111175
:101A30000CC02D853E85222011F060EA01C060E8CF
:101A40004F2DC3010E94630901C0812F62960FB61A
:101A5000F894DEBF0FBECDBFDF91CF911F910F91E4
:101A6000FF90EF90DF90CF90BF90AF909F908F90BE
:101A70007F906F905F904F903F902F9008958F923E
:101A80009F92AF92BF92CF92EF920F931F931F92AC
:101A90001F921F930F933F932F934901A12CB12CB9
:101AA000CC24C394E12C06E020E80E945F0C0F9048
:101AB0000F900F900F900F900F901F910F91EF903C
:101AC000CF90BF90AF909F908F9008958F929F92EC
:101AD000AF92BF92CF92EF92FF920F931F921F92FD
:101AE000FF92EF923F932F934901A12CB12C52E02A
:101AF000C52EE02E06E020E80E945F0C0F900F90AC
:101B00000F900F900F900F900F91FF90EF90CF904C
:101B1000BF90AF909F908F9008953F924F925F92A9
:101B20006F927F928F929F92AF92BF92CF92DF92ED
:101B3000EF92FF920F931F93CF93DF93CDB7DEB752
:101B4000C054D1090FB6F894DEBF0FBECDBF3C0123
:101B5000562E442E322EB02ECE0101966C017C0101
:101B6000022F29E030E0C3010E94660D81111BC0E5
:101B70008B809C801F93BF92DF92CF921F9280E454
:101B80008F93A12CB12C62E0C62EE32C06E020E856
:101B9000442D652DC3010E945F0C0F900F900F9094
:101BA0000F900F900F90C05CDF4F0FB6F894DEBF20
:101BB0000FBECDBFDF91CF911F910F91FF90EF909E
:101BC000DF90CF90BF90AF909F908F907F906F905D
:101BD0005F904F903F9008958F929F92AF92BF92E7
:101BE000CF92EF920F93CF931F921F921F921F924B
:101BF0001F921F92812C912CA12CB12CC12CE22E72
:101C000005E020E00E945F0CC82F6CE271E080E0EC
:101C100090E00E94E7160F900F900F900F900F909A
:101C20000F908C2FCF910F91EF90CF90BF90AF90EE
:101C30009F908F9008958F929F92AF92BF92CF9274
:101C4000EF920F931F921F921F921F921F921F924B
:101C5000812C912CA12CB12CC12CE22E09E020E08A
:101C60000E945F0C0F900F900F900F900F900F90AD
:101C70000F91EF90CF90BF90AF909F908F9008956D
:101C80008F929F92AF92BF92CF92DF92EF920F937B
:101C90001F93CF93DF9300D000D0CDB7DEB76C0198
:101CA000590148011C821B821A8219828E010F5F22
:101CB0001F4F9E012D5F3F4F0E94F508811109C003
:101CC00049815A816B817C8184019501C6010E9402
:101CD0007D0B0F900F900F900F90DF91CF911F9180
:101CE0000F91EF90DF90CF90BF90AF909F908F902B
:101CF0000895CF92DF92FF920F931F93CF93DF93BC
:101D000000D0CDB7DEB76C01662309F442C0062FC0
:101D100010E085E0689FB0011124F601E60FF71F7F
:101D20008085282F277086FF19C031E0E5E0FE2E60
:101D3000F601F39EE00DF11D1124808586958695B0
:101D4000869587708217E1F03F5F303188F3F601A6
:101D50008581821303C02150F601258385E0809F91
:101D6000F001819FF00D1124EC0DFD1D108681E026
:101D70008187128682E0C80ED11CD782C68209C034
:101D8000632FC6012A8339830E94790E2A81398103
:101D9000CFCF0F900F90DF91CF911F910F91FF90B8
:101DA000DF90CF900895CF93DF93EC016134A1F4DD
:101DB000FC01855B9F4F41E09E012E5F3F4F1586E2
:101DC00046871786348723873596E817F907B9F7CA
:101DD0001D82DF91CF9108950E94CC07682FCE011C
:101DE000DF91CF910C94790E0F931F93CF93DF93D4
:101DF000EC01022FCA3F8FEFD80711F486ED29C0FE
:101E00008E819F81892B01F12A87242F40E0CE010A
:101E10000E94DE07182F8823C9F0682FCE010E9488
:101E20005208009759F3FC010483212F40E060E041
:101E3000CE010E94EC0D082F882351F0612FCE01B6
:101E40000E94D30E802F05C087ED03C084ED01C032
:101E500080E0DF91CF911F910F9108952F923F92D3
:101E60004F925F926F927F928F929F92AF92BF92AA
:101E7000CF92DF92EF92FF920F931F93CF93DF9356
:101E8000CDB7DEB766970FB6F894DEBF0FBECDBFF5
:101E90007C01862E742E922E1B8A88E08C8B8CE31C
:101EA0008D8BD701ED91FC910190F081E02D60E0E8
:101EB000C70109956C01009709F4ABC0FC01A08033
:101EC000B180CE0143969183808394828E010F5F0F
:101ED0001F4F22E130E040E060E0C7010E943F0D6B
:101EE000D601AD92BC928111ACC029843A844B8456
:101EF0005C84BD81BE8B1E815701612C6501E6E5C6
:101F0000CE0ED11CD6018D919C91009789F1DC01F8
:101F1000ED91FC910084F185E02D0995811128C097
:101F2000F60180819181DC01ED91FC910088F189BD
:101F3000E02D612F09958823D9F0F60180819181E8
:101F4000DC01ED91FC910484F585E02DA201B10145
:101F50000995811160C0F60180819181DC01ED91CC
:101F6000FC910684F785E02D6E890995811153C097
:101F70006394B2E0AB0EB11CE0E16E12BFCF57012B
:101F8000612C6501F6E5CF0ED11CD6018D919C9197
:101F9000009789F1DC01ED91FC910084F185E02D41
:101FA0000995811128C0F60180819181DC01ED91B4
:101FB000FC910088F189E02D612F09958823B1F10A
:101FC000F60180819181DC01ED91FC910484F5851D
:101FD000E02DA201B101099581110DC0F6018081AA
:101FE0009181DC01ED91FC910684F785E02D6E89ED
:101FF00009958823D9F06394B2E0AB0EB11CE0E1FF
:102000006E12BFCF292D472D682DC7010E94F40EF7
:1020100018C086ED16C0092D272D482D662DC70145
:102020000E94CB09813D09F4A3CF0BC0092D272DB8
:10203000482D662DC7010E94CB09982F977F913DAF
:10204000D1F266960FB6F894DEBF0FBECDBFDF911A
:10205000CF911F910F91FF90EF90DF90CF90BF90A5
:10206000AF909F908F907F906F905F904F903F9038
:102070002F900895FF920F931F93CF93DF93EC015E
:1020800019990EC088EC0E94B30885FF05C0CE01E7
:102090000E94E80560E201C060E088EC0E94D1087F
:1020A0008091AC01813051F058F0823029F08330BA
:1020B00039F5FF24F3940DC0F12C0BC083E106C069
:1020C00080916102807F8031D9F081E1809361024B
:1020D00017C080916102807F803199F40E94B81608
:1020E00068537F4F8F4F9F4F60935D0270935E02E6
:1020F00080935F029093600280E28093610201C04E
:10210000F12C00E010E0FE01E00FF11FEA5AFF4F52
:1021100080819181009739F0DC01ED91FC9106807E
:10212000F781E02D09950E5F1F4F0032110559F719
:1021300080916102803409F446C070F4803269F104
:102140008033D9F1813109F088C0FE01EA58FF4F90
:10215000108200E010E00AC0813509F45AC08038CE
:1021600009F46AC0803509F078C03CC0FE01E00F78
:10217000F11FEA5AFF4F80819181009739F0DC010D
:10218000ED91FC910480F581E02D09950E5F1F4FC4
:102190000032110559F782E15EC00E94B816009125
:1021A0005D0210915E0220915F0230916002601B1F
:1021B000710B820B930B97FD50C061E088EE0E947B
:1021C000D10880E448C088EE0E94B30880FD45C075
:1021D00088ED0E94B308682F686088ED0E94D108DE
:1021E00080E539C088EC0E94B30886FF36C081E5DF
:1021F000809361020E94B8166C5E7F4F8F4F9F4F95
:1022000060935D0270935E0280935F029093600220
:1022100024C00E94B81600915D0210915E022091C8
:102220005F0230916002601B710B820B930B97FD74
:1022300014C080E8809361022F2D40E060E0CE0161
:102240000E942E0F882331F0823D39F08093620284
:1022500080EA01C080E980936102DF91CF911F91F4
:102260000F91FF9008958F929F92AF92BF92CF925D
:10227000EF920F93CF93DF93CDB7DEB7C054D10960
:102280000FB6F894DEBF0FBECDBF5F934F939E0194
:102290002F5F3F4F3F932F931F9220E42F9320E80F
:1022A000822E912C5B0132E2C32EE12C06E021E864
:1022B00040E0FC016681848195810E945F0C0F9053
:1022C0000F900F900F900F900F90C05CDF4F0FB6E4
:1022D000F894DEBF0FBECDBFDF91CF910F91EF908D
:1022E000CF90BF90AF909F908F9008958F929F92C4
:1022F000AF92BF92CF92EF920F93A62EB12C1F9266
:102300001F921F921F921F921F92812C912CC22EFE
:10231000E42E0AE021E240E0FC016681848195819F
:102320000E945F0C0F900F900F900F900F900F90E6
:102330000F91EF90CF90BF90AF909F908F900895A6
:102340008F929F92AF92BF92CF92EF920F93A62E51
:10235000B12C1F921F921F921F921F921F92812CCD
:10236000912CC12CE42E0BE021E240E0FC016681BF
:10237000848195810E945F0C0F900F900F900F90B9
:102380000F900F900F91EF90CF90BF90AF909F90D4
:102390008F9008950F931F93CF93DF93EC012A81C1
:1023A0002170F8018081982F9170291771F0E881D0
:1023B000F98180FF04C00680F781E02D03C004800E
:1023C000F581E02DB801CE0109952A81269521706D
:1023D000F801808181FB992790F9291771F0E88134
:1023E000F98181FF04C00284F385E02D03C00084DD
:1023F000F185E02DB801CE0109952A8122FB222723
:1024000020F9F801808182FB992790F9291771F052
:10241000E881F98182FF04C00684F785E02D03C0BE
:102420000484F585E02DB801CE010995F80181817C
:10243000811103C08281882341F0E881F981028003
:10244000F381E02DB801CE010995F80180818A83DE
:10245000DF91CF911F910F910895CF93DF93FC01EE
:10246000EA0180819181892B21F580E028C0888153
:102470009981892BD1F3DB018D919C91DC015C91D9
:10248000238130E0241B310980819181820F931FC9
:10249000DC015C93828181508283888199810197DC
:1024A00099838883DB018D919C91119701968D937F
:1024B0009C9342814111DBCF8381828381E0DF9154
:1024C000CF910895FC018285089581E0693009F07B
:1024D00080E00895CF93DF93EC018A819B81DC013A
:1024E000ED91FC910480F581E02D6A8509958A853E
:1024F000813439F4EA81FB81EA58FF4F808184609E
:1025000080831A861B861C861D861E861F86188A57
:1025100080E0DF91CF9108958F929F92AF92BF920A
:10252000CF92EF920F93A42EB12CB22A1F921F923A
:102530001F921F921F921F92812C912CC12CE62E6C
:1025400001E023E240E0FC016285828193810E94E8
:102550005F0C0F900F900F900F900F900F900F91B6
:10256000EF90CF90BF90AF909F908F9008958F92F3
:102570009F92AF92BF92CF92EF920F93A62EB12C63
:102580001F921F923F932F935F934F934A01C12C49
:10259000E12C00E023EA40E0FC0162858281938126
:1025A0000E945F0C0F900F900F900F900F900F9064
:1025B0000F91EF90CF90BF90AF909F908F90089524
:1025C0008F929F92AF92BF92CF92EF920F93A42ED1
:1025D000B12CB22A1F921F921F921F921F921F921C
:1025E000812C912CC12CE62E03E023E240E0FC017B
:1025F0006285828193810E945F0C0F900F900F90F3
:102600000F900F900F900F91EF90CF90BF90AF90E1
:102610009F908F9008952F923F924F925F926F926A
:102620007F928F929F92AF92BF92CF92DF92EF9262
:10263000FF920F931F93CF93DF93CDB7DEB7E99748
:102640000FB6F894DEBF0FBECDBF3C01362E242E50
:10265000DC011296ED90FC9013971A968C918111E3
:1026600003C1D701ED91FC910190F081E02D60E074
:10267000C70129AF09956C0129AD009709F4F6C08F
:10268000FC01A080B180A114B10409F4F1C04301A0
:10269000F4E08F0E911CDC0111969C928E921496A0
:1026A0002C93FE0131962F018F0128E030E040E0AD
:1026B00060E0D30112968D919C9113970E943F0D7B
:1026C000F60114828111DAC019818D81893009F0F7
:1026D000D1C0D701ED91FC910280F381E02D222D34
:1026E00041E0632DC7010995F3018287882309F42E
:1026F000C3C098859583282F40E060E08281938154
:102700000E94EC0D082F882391F0D601AD92BC9267
:10271000D701ED91FC910480F581E02DD3011A964B
:102720006C91C7010995F3011286102FABC01132CD
:1027300008F010E2D601AD92BC9211110BC09401C9
:1027400042E0F3016285828193810E948D088111AC
:1027500098C011C0212F30E0820140E0D3011A96C9
:102760006C911A9712968D919C9113970E943F0D30
:10277000811187C0E4CF1F921F925F924F921F92E8
:1027800088E08F9388E0882E912CA12CB12C99E2BF
:10279000C92EE12C06E020EA40E0F3016285828147
:1027A00093810E945F0C182F0F900F900F900F9045
:1027B0000F900F90811166C08B81D3011B968C9373
:1027C0001B97720100E028E030E040E01A966C911F
:1027D0001A9712968D919C9113970E94660D811104
:1027E00050C02B813C8140E0F3016285828193815E
:1027F0000E94660D811145C0298130E0CE0181968D
:102800007C0140E0D3011A966C911A9712968D9133
:102810009C9113970E94660D811133C02E8140E078
:10282000F3016285828193810E941B0E811129C070
:1028300001E0D3011B968C911B97801740F020E09C
:10284000402F68E0C3010E94E0120F5FF2CF1296A2
:10285000ED91FC911397EA58FF4F8081846080834B
:1028600081E050968C930EC019ED0CC016ED0AC095
:1028700017ED08C011ED06C014ED04C0F601B182D9
:10288000A082182F812FE9960FB6F894DEBF0FBEF5
:10289000CDBFDF91CF911F910F91FF90EF90DF900F
:1028A000CF90BF90AF909F908F907F906F905F90F0
:1028B0004F903F902F900895BF92CF92DF92EF926A
:1028C000FF920F931F93CF93DF9300D000D0CDB72B
:1028D000DEB77C01B62E19821A821B821C8220E090
:1028E000462F61E10E948C1220E04B2D60E1C70170
:1028F0000E948C1220E04B2D64E0C7010E94E01280
:1029000023E0C22ED12C9E012F5F3F4F44E050E0C8
:102910006B2DC7010E94B712882301F120E04B2DD7
:1029200064E1C7010E948C1220E04B2D60E1C701D9
:102930000E948C1264E170E080E090E00E94E71653
:102940000F900F900F900F90DF91CF911F910F91EB
:10295000FF90EF90DF90CF90BF90089509811A818A
:102960002B813C811D7F0330114020413105B1F2A4
:1029700064E670E080E090E00E94E71681E0C81A0B
:10298000D10809F0C0CFCACFCF93DF93FC018BE70A
:1029900091E0918380837383628312861386148609
:1029A000158616861786108A148288E085839CE334
:1029B000968391E09783808784E081876115710514
:1029C000B9F0CB01A0E0B0E0EC01CA5ADF4F28819A
:1029D0003981232B41F49B96AA0FBB1FA60FB71F6B
:1029E000ED93FC9305C011960296A031B10561F7F5
:1029F000DF91CF910895DF92EF92FF920F931F9393
:102A0000CF93DF93EC01D62E7A01FA010081118178
:102A1000228133810130F3E01F07F1E02F073105F8
:102A2000D1F060F40115E1E01E072E07310571F1C8
:102A3000013011402140310571F062C0033081E066
:102A4000180780E128073105E1F1033013402041E8
:102A50003105B9F155C080916302811151C020E068
:102A60004D2D61E1CE010E948C1220E04D2D60E1E0
:102A7000CE010E948C1220E04D2D64E0CE010E9418
:102A8000E01281E08093630281EB3BC020E0462F9F
:102A900061E1CE010E948C1220E04D2D60E1CE015B
:102AA0000E948C12109263026A8567708D2D877068
:102AB000660F660F660F682B8A819B810E947D07D7
:102AC0001FC020E04D2D64E1CE010E948C1220E059
:102AD0004D2D60E1CE010E948C1264E170E080E037
:102AE00090E00E94E7166A85F70121812695217002
:102AF00067704D2D8A819B810E942E0F1092630278
:102B000080E0DF91CF911F910F91FF90EF90DF90C8
:102B10000895CF92DF92EF920F931F93CF93DF939D
:102B2000CDB7DEB72E970FB6F894DEBF0FBECDBF80
:102B30006C0181E090E09E878D87E12C8E010F5F14
:102B40001F4F9E01235F3F4F41E0F6016285828166
:102B500093810E94400E811151C002E011E08981F1
:102B60008023D1F019861A861B861C869E01275F5A
:102B70003F4F44E050E0612FC6010E94B71281111F
:102B80000BC0AE01475F5F4F612FC6010E94FB146F
:102B9000813B99F1811132C0000F1F5F1830F9F6A7
:102BA00011E0F6018385811740F119861A861B868C
:102BB0001C869E01275F3F4F44E050E0612FC60115
:102BC0000E94B712811117C089859A85877091700C
:102BD0008130914081F48B859C8581609C878B87B7
:102BE000AE01475F5F4F612FC6010E94FB14813B1E
:102BF00021F0811103C01F5FD4CF80E02E960FB665
:102C0000F894DEBF0FBECDBFDF91CF911F910F9122
:102C1000EF90DF90CF9008950F931F93CF93DF93A2
:102C2000EC0188898823F1F00E94B8160C851D8577
:102C30002E853F85601B710B820B930B97FD0FC098
:102C4000CE010E948915182F0E94B8166C597F4F2B
:102C50008F4F9F4F6C877D878E879F8701C010E0C5
:102C6000812F01C080E0DF91CF911F910F910895D6
:102C7000CF93CFB7F89480916702811127C0EAE91A
:102C8000F0E08491E6E8F0E09491E82FF0E0EE0FB8
:102C9000FF1FE255FF4FA591B4918C91892321F438
:102CA00061E08AE00E94C91761E08AE00E94901703
:102CB0008CB580618CBD8CB580648CBD61E08DE08D
:102CC0000E94901761E08BE00E949017809167024C
:102CD0008F5F80936702CFBFCF9108951F920F92AD
:102CE0000FB60F9211242F933F938F939F93AF931F
:102CF000BF938091690290916A02A0916B02B0919A
:102D00006C023091680223E0230F2D3720F40196E6
:102D1000A11DB11D05C026E8230F0296A11DB11DFE
:102D2000209368028093690290936A02A0936B02D9
:102D3000B0936C0280916D0290916E02A0916F022F
:102D4000B09170020196A11DB11D80936D02909308
:102D50006E02A0936F02B0937002BF91AF919F91EA
:102D60008F913F912F910F900FBE0F901F9018954C
:102D70002FB7F8946091690270916A0280916B029A
:102D800090916C022FBF08953FB7F89480916D0227
:102D900090916E02A0916F02B091700226B5A89B2F
:102DA00005C02F3F19F00196A11DB11D3FBF662739
:102DB000782F892F9A2F620F711D811D911D42E07E
:102DC000660F771F881F991F4A95D1F708958F9234
:102DD0009F92AF92BF92CF92DF92EF92FF926B01E0
:102DE0007C010E94C4164B015C01C114D104E104B2
:102DF000F104F1F00E9408190E94C41668197909BB
:102E00008A099B09683E73408105910570F321E0B2
:102E1000C21AD108E108F10888EE880E83E0981EF6
:102E2000A11CB11CC114D104E104F10429F7DDCFC8
:102E3000FF90EF90DF90CF90BF90AF909F908F90DA
:102E400008958230910538F0880F991F880F991FD7
:102E500005970197F1F70895789484B5826084BD51
:102E600084B5816084BD85B5826085BD85B581608E
:102E700085BDEEE6F0E0808181608083E1E8F0E0EE
:102E80001082808182608083808181608083E0E81D
:102E9000F0E0808181608083E1EBF0E080818460FC
:102EA0008083E0EBF0E0808181608083EAE7F0E0FE
:102EB0008081846080838081826080838081816062
:102EC00080838081806880831092C1000895833060
:102ED00081F028F4813099F08230A1F00895873094
:102EE000A9F08830B9F08430D1F4809180008F7DD2
:102EF00003C0809180008F7780938000089584B50F
:102F00008F7702C084B58F7D84BD08958091B00015
:102F10008F7703C08091B0008F7D8093B0000895BB
:102F2000CF93DF9390E0FC01E458FF4F2491FC0124
:102F3000E057FF4F8491882349F190E0880F991F53
:102F4000FC01E255FF4FA591B4918C559F4FFC01B8
:102F5000C591D4919FB7611108C0F8948C912095C8
:102F600082238C93888182230AC0623051F4F894C2
:102F70008C91322F309583238C938881822B888388
:102F800004C0F8948C91822B8C939FBFDF91CF91DA
:102F900008950F931F93CF93DF931F92CDB7DEB7A2
:102FA000282F30E0F901E859FF4F8491F901E458E6
:102FB000FF4F1491F901E057FF4F04910023C9F02E
:102FC000882321F069830E9467176981E02FF0E070
:102FD000EE0FFF1FEC55FF4FA591B4919FB7F894EA
:102FE0008C91611103C01095812301C0812B8C93BA
:102FF0009FBF0F90DF91CF911F910F9108951F9266
:103000000F920FB60F9211242F938F939F93EF93EC
:10301000FF93E0918102F09182028081E09187022A
:10302000F091880282FD12C0908180918A028F5FA8
:103030008F7320918B02821751F0E0918A02F0E0A9
:10304000EF58FD4F958F80938A0201C08081FF91D8
:10305000EF919F918F912F910F900FBE0F901F9026
:1030600018951F920F920FB60F9211242F933F9332
:103070004F935F936F937F938F939F93AF93BF9380
:10308000EF93FF9381E792E00E944419FF91EF9143
:10309000BF91AF919F918F917F916F915F914F9170
:1030A0003F912F910F900FBE0F901F90189581E7C1
:1030B00092E00E94091921E0892B09F420E0822F77
:1030C0000895109274021092730288EE93E0A0E0CB
:1030D000B0E08093750290937602A0937702B0934C
:1030E000780280EA91E0909372028093710285ECFD
:1030F00090E090937E0280937D0284EC90E0909328
:10310000800280937F0280EC90E090938202809313
:10311000810281EC90E0909384028093830282ECA0
:1031200090E0909386028093850286EC90E09093E5
:1031300088028093870210928A0210928B0210926A
:103140008C0210928D020895CF92DF92EF92FF923F
:103150000F931F93CF93DF937C016A01EB0100E093
:1031600010E00C151D0571F06991D701ED91FC91EE
:103170000190F081E02DC7010995892B19F00F5FAF
:103180001F4FEFCFC801DF91CF911F910F91FF909B
:10319000EF90DF90CF9008956115710581F0DB010C
:1031A0000D900020E9F7AD0141505109461B570B26
:1031B000DC01ED91FC910280F381E02D099480E027
:1031C00090E008956DE871E00C94CC180F931F9374
:1031D000CF93DF93EC010E94CC188C01CE010E94AA
:1031E000E218800F911FDF91CF911F910F910895E9
:1031F00008950E942C170E94F8180E946206C6E3E8
:10320000D9E10E949A052097E1F30E943619F9CF7F
:103210000895FC01818D228D90E0805C9F4F821B80
:1032200091098F7399270895FC01918D828D9817CC
:1032300031F0828DE80FF11D858D90E008958FEFBC
:103240009FEF0895FC01918D828D981761F0828D1A
:10325000DF01A80FB11D5D968C91928D9F5F9F73CA
:10326000928F90E008958FEF9FEF089587E598E1A2
:10327000892B49F080E090E0892B29F00E945718B3
:1032800081110C9400000895FC01848DDF01A80FCA
:10329000B11DA35ABF4F2C91848D90E001968F737E
:1032A0009927848FA689B7892C93A089B1898C919D
:1032B00080648C93938D848D981306C00288F38963
:1032C000E02D80818F7D80830895CF93DF93EC0183
:1032D000888D8823C9F0EA89FB89808185FD05C036
:1032E000A889B9898C9186FD0FC00FB607FCF5CF70
:1032F000808185FFF2CFA889B9898C9185FFEDCFB8
:10330000CE010E944419E7CFDF91CF910895CF926B
:10331000DF92FF920F931F93CF93DF931F92CDB74E
:10332000DEB76C0181E0D60158968C9358975B9676
:103330009C915B975C968C915C97981307C0509614
:10334000ED91FC915197808185FD2EC0F601038D92
:1033500010E00F5F1F4F0F731127F02EF601848DC1
:10336000F81211C00FB607FCF9CFD6015096ED91B7
:10337000FC915197808185FFF1CFC60169830E943E
:1033800044196981EBCF838DE80FF11DE35AFF4F9C
:103390006083D6015B960C935B975296ED91FC91FE
:1033A0005397808180620CC0D6015696ED91FC91B6
:1033B000579760835096ED91FC915197808180647E
:1033C000808381E090E00F90DF91CF911F910F916A
:1033D000FF90DF90CF900895AA1BBB1B51E107C05F
:1033E000AA1FBB1FA617B70710F0A61BB70B881F95
:1033F000991F5A95A9F780959095BC01CD01089524
:1034000097FB072E16F4009407D077FD09D00E9491
:10341000EC1907FC05D03EF4909581959F4F0895D7
:10342000709561957F4F0895EE0FFF1F0590F49101
:10343000E02D0994DC0101C06D9341505040E0F74C
:063440000895F894FFCF8F
:1034460000000E0380000C000100320000000400A2
:103456000200010003004F534320646964206E6F2D
:10346600742073746172742E00000000004D020017
:103476000000002A0100000000CA1135012B0130AE
:10348600018F009000AF00B0000000000026048805
:1034960000BA00B803D5008A008B00D800DD00E230
:1034A60000B100EA00ED00FEFF0000200100000070
:1034B600005208DE07D30E000000000B1388006AD6
:1034C600120C1662125C148B0065128D000D0A0038
:1034D6006E616E00696E66006F7666000000000021
:0C34E6008719A418091922191419651976
:00000001FF
